:1000000049C07BC060C05FC05EC05DC05CC05BC0FB
:100010005AC059C058C057C056C055C054C053C02C
:1000200052C051C050C009022200010100807D0968
:100030000400000103000000092101010001221653
:10004000000705810308000A1201100100000008E2
:10005000C016DF0500010102000110034C0045003D
:100060004400430075006200650010034300540023
:1000700048004E002E0064006500040309040600D9
:10008000FF0901A101150026FF007508950109006F
:10009000B20201C011241FBECFEDCDBF10E0A0E61B
:1000A000B0E0E2ECF7E002C005900D92A436B10793
:1000B000D9F710E0A4E6B0E001C01D92AF39B10756
:1000C000E1F755D17CC39CCFA82FB92F80E090E0F9
:1000D00041E050EA609530E009C02D918227979564
:1000E000879510F084279527305EC8F36F5FA8F3DB
:1000F0000895EADF8D939D930895CF93CFB7CF9363
:10010000C395819BE9F7819B09C0819B07C0819BB7
:1001100005C0819B03C0819B01C0A3C0DF93C09138
:100120008200DD27C757DF4F819B02C0DF91EBCFF5
:100130002F930F931F9300B32FEF01FB20F94F93E1
:100140003F9310B34FEF012701FB21F93BE031C092
:100150004E7F012F10B3216028C0102F4D7F2260E9
:10016000000000B329C04B7F2460012F000010B3B2
:100170002BC010B3477F28602AC04F7E00B3206198
:100180002CC04F7D10B320622FC04F7B00B3206482
:1001900032C0422700B349934FEF0000102711FBF4
:1001A00020F910B31670C9F1297F91F2012701FBE4
:1001B00021F900B3237F89F2315058F1102711FB48
:1001C00022F910B3277E79F2012701FB23F92F7C56
:1001D00081F200B3102711FB24F92F7971F200C0CE
:1001E00010B3012701FB25F92F7359F200C000B3AA
:1001F000102711FB26F9223040F200C010B301276E
:1002000001FB27F9243028F64F77206810B300004F
:10021000F9CF10E41ABF002719C03B503195C31B1A
:10022000D04010E41ABF0881033CF9F00B34E9F028
:10023000209180001981110F1213EDCF4A81441FC4
:10024000093641F10D3211F0013E29F70093870084
:100250003F914F911F910F912F91DF91CAB7C6FD2A
:100260004FCFCF91CFBFCF911895209187002223F8
:1002700079F310918500112369F534306AF13093D8
:10028000850020938100109182003BE0311B309368
:10029000820022C0009185000130E4F40AE54F702D
:1002A00049F43091620034FD19C000936200C9E640
:1002B000D0E018C03091740034FD10C00093740079
:1002C000C5E7D0E00FC02795A8F45150A9F4220F3C
:1002D0000000F9CF4AE503C042ED01C0432FC4E15D
:1002E000D0E032E011B31660919A11BB02B320E462
:1002F00016E05F93012756E002BB279520F451508A
:1003000021F4220FF9CF012756E000003B5A02BB2F
:10031000D0F2279528F4515029F4220F0000F9CF8C
:10032000012756E0279502BB20F4515021F4220FFB
:10033000F9CF012756E02991332302BB21F6097F2B
:1003400010918600110FC651D04002BB11F01093DE
:10035000800010E41ABF026011B3197F402F497F5B
:100360005F9100C000C002BB11BB42BB71CF8FEFD9
:1003700087BB88BB88E781BB80E482BB81E792E0D2
:100380009BBD8ABD8BE08EBD7894DED166D008B669
:1003900006FEFCCF80E488BFF894115011F58091DF
:1003A0006000D03229F48130C1F41092600015C091
:1003B0008823A1F08D2F90E0880F991F880F991F37
:1003C00080509040D4D16093650070936600809314
:1003D000670090936800DF5F01C0D0E01091680073
:1003E000187F82B3837C82BB8C2F69E0B7D1282F22
:1003F00040916500509166006091670070916800BF
:1004000004C076956795579547958A95D2F740959C
:1004100048BB8091650090916600A0916700B09103
:10042000680004C0B695A795979587952A95D2F749
:1004300090FF02C0969801C0969A22B388E090E09F
:100440000C2E01C0880F0A94EAF7822B82BBCF5F83
:10045000C33009F4C0E0789499CFCF93DF938091B3
:100460008500835087FDA3C0909182002091810078
:100470002D3209F09AC0883009F097C0CCE0D0E066
:10048000C91BD109C757DF4F83EC809369008AE508
:1004900080936200109264008881807619F0CE010A
:1004A000E7D07AC09A81109272008981811106C0CA
:1004B0001092730022E730E082E06AC0853019F4C0
:1004C0009093860062C0863009F049C08B818130EC
:1004D00041F488E490E0909384008093830082E16B
:1004E0003AC0823041F486E290E090938400809399
:1004F000830082E230C08330C9F4911108C08AE7DA
:1005000090E0909384008093830084E024C0913035
:1005100019F48AE690E004C09230E1F48AE590E0B4
:10052000909384008093830080E115C0813241F470
:1005300088E390E0909384008093830089E00BC06F
:10054000823241F48EE790E09093840080938300A0
:1005500086E101C080E090E4909364001DC0883083
:1005600069F0893019F4909388000FC08A3049F0FF
:100570008B3059F48BE48093750007C028E830E095
:1005800002C022E730E081E003C022E730E080E0F3
:1005900030938400209383009F81911104C09E8139
:1005A000981708F4892F809361001092850080913C
:1005B000620084FF43C0809161008F3F09F43EC018
:1005C000C82F893008F0C8E08C1B8093610090919F
:1005D000690088E8892780936900CC2319F180910C
:1005E000830040918400209164009C2F980F26FF87
:1005F0000AC0AAE6B0E0E82FF42F84918D933196DB
:100600009E13FBCF0BC02AE630E0A82FB42F8D91AC
:10061000F90181939F01FD019A13F9CFF0938400B2
:10062000E09383006C2F8AE690E063DDCC5FCC30F2
:1006300019F08FEF80936100C093620084E190B362
:10064000967031F48150D9F7109286001092800094
:10065000DF91CF91089585B7826085BF8BB78064A5
:100660008BBFE4E7F0E08BE481838AE58083089523
:100670000F931F93FC0180818076803409F060C065
:100680008181813009F043C084814091650050919F
:100690006600609167007091680081111AC08281C4
:1006A000038110E0102F0027080F111D222717FDCE
:1006B0002095322F44275527042B152B262B372B1B
:1006C00000936500109366002093670030936800E4
:1006D00037C022819381892F90E0982F8827820F3D
:1006E000911DAA2797FDA095BA2FDC01992788278D
:1006F00066277727842B952BA62BB72B8093650035
:1007000090936600A0936700B093680019C0823090
:1007100091F440916500509166006091670070917E
:100720006800848190E0880F991F880F991F80507E
:10073000904020D005C0833019F4828180936000FE
:1007400080E01F910F910895CF9385DF899AC15062
:1007500011F00000FCCF8998CF910895002480FD0E
:10076000060E660F11F08695D1F7802D0895A6E14B
:1007700044E00AC0242F16D0252F14D000C011D079
:10078000272F10C0A82F862FE82FE199FECF1FBA80
:1007900005C0EEBBE09AE3950DB20D924150C8F74B
:1007A0000895262FE199FECF1CBA1FBA8EBB2DBB30
:1007B0000FB6F894E29AE19A0FBE01960895F89464
:0207C000FFCF69
:0407C20002FF5A00D8
:00000001FF
